:0A19F80000010202030304040505C8
:10080C00E4F558F557F556F555C203C200C202C2BD
:10081C00011209E47E007F908E0A8F0B7512007511
:10082C0013A27508007509AC7510007511DA7514F2
:10083C000175150890E680E030E70E85080C8509F7
:10084C000D85100E85110F800C85100C85110D85F2
:10085C00080E85090FEE54E0700302097D755900EE
:10086C00755A807E007F908E5B8F5CC3742E9FFFC9
:10087C0074019ECF2402CF3400FEE48F548E53F5C6
:10088C0052F551F550F54FF54EF54DAF54AE53AD05
:10089C0052AC51AB50AA4FA94EA84DC3120BF050FD
:1008AC002AE55A2550F582E559354FF58374CDF07C
:1008BC00E4FAF9F8E5502401F550EA354FF54FE923
:1008CC00354EF54EE8354DF54D80C0E4F550F54FFD
:1008DC00F54EF54DAF54AE53AD52AC51AB50AA4F93
:1008EC00A94EA84DC3120BF05035AE4FAF50E55C7E
:1008FC002FF582E55B3EF583E0FDE55A2FF582E5A9
:10090C00593EF583EDF0E4FAF9F8EF2401F550EADD
:10091C003EF54FE9354EF54EE8354DF54D80B58534
:10092C00590A855A0B74902480FF740034FFFEC35F
:10093C00E5139FF513E5129EF512C3E50D9FF50D1A
:10094C00E50C9EF50CC3E50F9FF50FE50E9EF50E1D
:10095C00C3E5099FF509E5089EF508C3E5119FF568
:10096C0011E5109EF510C3E5159FF515E5149EF5E0
:10097C0014D2E843D82090E668E04409F090E65C95
:10098C00E0443DF0D2AF90E680E020E105D20812C1
:10099C0011CF90E680E054F7F0538EF8C20330018B
:1009AC0005120572C20130032912008E5024C203B5
:1009BC001218A220001690E682E030E704E020E155
:1009CC00EF90E682E030E604E020E0E41217D0126B
:0709DC0011FE1214E080C7B8
:0109E30022F1
:1005720090E6B9E0700302064E1470030206F724F7
:10058200FE700302078C24FB7003020648147003FA
:1005920002064214700302063614700302063C245B
:1005A2000560030207F8121A88400302080490E665
:1005B200BBE024FE602C14604724FD6016146031F9
:1005C20024067066E50A90E6B3F0E50B90E6B4F017
:1005D200020804E51290E6B3F0E51390E6B4F002E7
:1005E2000804E50C90E6B3F0E50D90E6B4F00208DD
:1005F20004E50E90E6B3F0E50F90E6B4F0020804CD
:1006020090E6BAE0FF1217FCAA06A9077B01EA49A5
:100612004B600DEE90E6B3F0EF90E6B4F002080402
:1006220090E6A0E04401F002080490E6A0E0440154
:10063200F00208041219C3020804121A480208043C
:100642001216330208041219B1020804121A8A405F
:100652000302080490E6B8E0247F602B14603C2477
:100662000260030206EDA200E433FF25E0FFA202CE
:10067200E4334F90E740F0E4A3F090E68AF090E68E
:100682008B7402F0020804E490E740F0A3F090E6D5
:100692008AF090E68B7402F002080490E6BCE05403
:1006A2007EFF7E00E0D3948040067C007D018004C2
:1006B2007C007D00EC4EFEED4F24F8F58274193E6D
:1006C200F583E493FF3395E0FEEF24A1FFEE34E6D9
:1006D2008F82F583E0540190E740F0E4A3F090E6C6
:1006E2008AF090E68B7402F002080490E6A0E044DF
:1006F20001F0020804121A8C400302080490E6B8C2
:10070200E024FE601D2402600302080490E6BAE0C1
:10071200B40105C20002080490E6A0E04401F00220
:10072200080490E6BAE0705990E6BCE0547EFF7E81
:1007320000E0D3948040067C007D0180047C007D33
:1007420000EC4EFEED4F24F8F58274193EF583E479
:1007520093FF3395E0FEEF24A1FFEE34E68F82F59E
:1007620083E054FEF090E6BCE05480FF1313135470
:100772001FFFE0540F2F90E683F0E04420F00208C0
:100782000490E6A0E04401F08078121A8E50739033
:10079200E6B8E024FE60202402706790E6BAE0B476
:1007A2000104D200805C90E6BAE06402605490E6F4
:1007B200A0E04401F0804B90E6BCE0547EFF7E0056
:1007C200E0D3948040067C007D0180047C007D00A3
:1007D200EC4EFEED4F24F8F58274193EF583E49356
:1007E200FF3395E0FEEF24A1FFEE34E68F82F5831E
:1007F200E04401F0800C120130500790E6A0E04482
:0908020001F090E6A0E04480F052
:01080B0022CA
:03003300021A743A
:041A740053D8EF3222
:1000900012010002000000401816111100000102B8
:1000A00000010A06000200000040010009022E00C3
:1000B000010100A0FA0904000004FF000000070588
:1000C0000102400000070586020002000705020247
:1000D0000002000705810240000009022E00010114
:1000E00000A0FA0904000004FF0000000705010257
:1000F000400000070586024000000705020240009C
:100100000007058102400000040309040E035100AA
:1001100048005900430043004400140351004800C4
:1001200059002D0031003100530020002000000054
:03004300021200A6
:0300530002120096
:101200000219270002199B000219850002193F00EC
:1012100002166A000216A100021A9000021A91003A
:10122000021A9200021A93000217A3000210630030
:10123000021A9400021A9500021A9600021A9700E8
:10124000021A9800021A9100021A9900021A9A00D2
:10125000021A9B00021A9C00021A9D00021A9E00AC
:10126000021A9F00021A9100021A9100021A9100BC
:10127000021AA000021AA100021AA200021AA30078
:10128000021AA400021AA500021AA600021AA70058
:10129000021AA800021AA900021AAA00021AAB0038
:1012A000021AAC00021AAD00021AAE00021AAF0018
:0812B000021AB000021AB1009D
:1017D00090E682E030E004E020E60B90E682E03024
:1017E000E119E030E71590E680E04401F07F147ED7
:0C17F000001215B590E680E054FEF022D7
:1018A20090E682E044C0F090E681F04387010000B8
:0418B2000000002210
:1011CF0030080990E680E0440AF0800790E680E05E
:1011DF004408F07FDC7E051215B590E65D74FFF0D4
:0F11EF0090E65FF05391EF90E680E054F7F02226
:0217FC00A9073B
:1017FE00AE14AF158F828E83A3E064037017AD0114
:10180E0019ED7001228F828E83E07C002FFDEC3E5D
:09181E00FEAF0580DF7E007F00B3
:01182700229E
:1015B5008E638F6490E600E054187012E564240190
:1015C500FFE43563C313F563EF13F564801590E607
:1015D50000E05418FFBF100BE56425E0F564E563F2
:1015E50033F563E5641564AE63700215634E6005FB
:0615F5001218B680EE2280
:1018B6007400F58690FDA57C05A3E582458370F945
:0118C60022FF
:1014600042274D000042274200004227440000412D
:10147000270000412701004127460041274C000179
:101480003A00044800000000042E0000C350022C63
:101490001A000227000002420000024503F7023C46
:1014A000000002240000022A00000134010139007A
:1014B0000138000141000144000137000232000000
:1014C000014CA00136000123000140000129000168
:0F14D0003B00C107014700012200013E00C1049B
:0B19E20030080453B1EF2243B1102283
:1018EB008E648F65E565456460177FCB7E011219A9
:1018FB0057000000000000E5651565700215648057
:02190B00E322D5
:0B19ED00AF3A90274DE4F0A3EFF0228A
:100EBA00E4F564F565FDFC902748E0FEA3E07A00BE
:100ECA002400F565EA3EF564902700E0FEA3E024DD
:100EDA0000FDEA3EFCC3E5659DFFE5649CFE9027A4
:100EEA0042F0A3EFF0902745E02FF0902744E03E30
:100EFA00F0D3A3E094D0902744E06480948740071D
:100F0A007407F0A374D0F0C3902745E0943090277B
:100F1A0044E064809478500774F8F0A37430F09039
:100F2A002744E0FEA3E07802C333CE33CED8F9FFDC
:100F3A007C007D0A120BA4AA06AB07902742E0FEAA
:100F4A00A3E0FF7C007D0F120B92EF2BFFEE3AFE1F
:100F5A0090274DF0A3EFF0D394FFEE648094804085
:100F6A000990274DE4F0A374FFF0C390274DE06485
:100F7A008094805004E4F0A3F090274DE0FEA3E0B3
:100F8A00FF7C007D02120BA490274DEEF0A3EFF038
:010F9A002234
:1011280090274CE0B4011FAD357F42121853902729
:101138004EE0FD7F4E121853E4FD7F90121853E4E1
:1011480090274CF0807390E678E04480F090E67940
:101158007491F07F647E0012195790E679E0902729
:1011680047F07F647E0012195790E679E09027488F
:10117800F07F647E0012195790E679E0902749F0D5
:101188007F647E0012195790E679E090274AF09024
:10119800E678E04440F0902748E090E7C1F09027D7
:1011A80049E090E7C2F090274EE0FFC3747F9F901C
:1011B800E7C3F090274C7401F0902746E0600412D2
:0711C8000EBA221219ED22FC
:1009E40090E6007412F090E6017443F00000009069
:1009F400E61074A0F000000000000090E611F00082
:100A0400000000000090E612F0000000E490E613FD
:100A1400F000000090E61474E0F0000000E490E6BA
:100A240015F000000090E6047480F00000007402E9
:100A3400F00000007406F0000000E4F000000090F4
:100A4400E60274E6F000000090E60374F8F000009B
:100A54000090E670E04440F0000000E490E609F005
:100A640000000053B2FE43B20243B20890E61804F9
:100A7400F00000007411F000000090E61A7409F010
:100A8400000000E490E671F090E672F075B4FF7532
:100A9400B6BF90E65EE04408F0000000E490E68D06
:100AA400F090E65EE04404F0000000E490E68FF08D
:100AB400C2081219E2D281121A6DE4FD7F8012136A
:100AC400D97F647E001215B57D807F801213D9C250
:100AD400057D0D7F401213D97D787F201213D9E450
:100AE400FD7F101213D9E4FD7F081213D97D0F7F07
:100AF400021213D9E4FD7F041213D9121A5090E69E
:100B04007AE054FEF0E4FD7F901218537F647E0077
:100B14001215B57DFF7F421218537F647E001215B3
:100B2400B57DAF7F4E121853121AB275B6BF1218A4
:0F0B340028D2A053B17F12196E7F341219D52227
:1014E000E4FAF9F8E54B2401F54BEA354AF54AE907
:1014F0003549F549E83548F548AF31AE30AD2FAC48
:101500002EAB4BAA4AA949F8C3120BF0700C12116A
:1015100028E4F54BF54AF549F548300715753E01C5
:10152000E540B40105E5B120E6F6120C7CC207E403
:10153000F53E0522D3E5229400748094884003E4AC
:0D154000F522E522700412190D22D2A0221E
:02008E00D3227B
:0211FE00D322FA
:021A8800D32267
:1016330090E680E030E71590E6247402F0000000A5
:10164300E490E625F0000000D2058013E490E62440
:10165300F000000090E6257440F0000000C2059001
:07166300E6BAE0F53FD322D7
:1019B10090E740E53FF0E490E68AF090E68B04F092
:0219C100D3222F
:081A480090E6BAE0F526D32276
:1019C30090E740E526F0E490E68AF090E68B04F099
:0219D300D3221D
:021A8A00D32265
:021A8C00D32263
:021A8E00D32261
:1001300090E6B9E0120C010156B301A3B50380B6F5
:1001400003BBC003DBC10459C204A0C50503C60537
:1001500034C70000056EE490E68AF090E68BF090DC
:10016000E6A0E020E1F990E68BE0F55D000000906C
:10017000E6047480F000000053297FAD29FF1213BC
:10018000D990E6047406F0000000E4F07F0AFE1245
:1001900015B5432980AD297F801213D9D207C2A09B
:1001A000020570E490E68AF090E68BF090E6A0E01D
:1001B00020E1F990E68BE0F55DD3943F4024E4F52F
:1001C0005E7440255EF582E434E7F583E0FF740257
:1001D000255EF582E43427F583EFF0055EE55EB435
:1001E00040DF7F9A7E00121A02902702E0FF7E0015
:1001F000121A0C902702E0FF7E00121A16902702B6
:10020000E0FF7E00121A20902703E075F004A4FF9F
:10021000AEF0121A2A902703E075F004A4FFAEF0A6
:10022000121A34902703E075F004A4FFAEF0121AFE
:100230003E902707E0C3940250035329CF9027072D
:10024000E0B40208E52954CF2410F529902707E0EF
:10025000B40308E52954CF2420F529902707E0B4FA
:100260000408E52954CF2430F529902723E07003B2
:100270005329B7902723E0B40108E529444054F7F7
:10028000F529902723E0B40208E52954BF4408F576
:1002900029902728E070055329FD80034329029007
:1002A0002709E0FD7F401213D990270AE0FD7F2047
:1002B0001213D9902713E0FD7F101213D990271441
:1002C000E0FD7F081213D9902725E0F53990272209
:1002D000E0F538902726E0F541902730E0F537909B
:1002E0002735E0F536A3E0F54490273CE0F54C9047
:1002F0002708E0F534E534700375340190270DE0EC
:10030000FEA3E07C002400F528EC3EF527A3E0FEE8
:10031000A3E02400F543EC3EF542902709E0FEA35C
:10032000E02400F52DEC3EF52CA3E0FEA3E0240034
:10033000F546EC3EF545902713E0FEA3E02400F5DA
:100340003DEC3EF53C902711E0FEA3E02400F52BA8
:10035000EC3EF52A902731E0FEA3E02400F525ECE1
:100360003EF52490271FE0FD7F021213D99027202D
:10037000E0FD7F041213D9902741E0F54702057094
:10038000E4F55E7402255EF582E43427F583E0FF30
:100390007440255EF582E434E7F583EFF0055EE511
:1003A0005EB440DF000000E490E68AF000000090B8
:1003B000E68B7440F0121828020570A298E433907E
:1003C000E740F0A3E599F0000000E490E68AF00031
:1003D000000090E68B7402F0020570E490E68AF06B
:1003E00090E68BF090E6A0E020E1F990E68BE0F556
:1003F0005DC298D39400500302057090E740E094EA
:100400000A5007E02430FF1219D590E740E0B40A03
:10041000057F611219D590E740E0B40B057F6212A9
:1004200019D590E740E0B40C057F631219D590E729
:1004300040E0B40D057F641219D590E740E0B40E9A
:10044000057F651219D590E740E0640F600302054F
:10045000707F661219D502057090E7407411F0A301
:10046000740CF0A304F0A37478F0A3740AF0A374DE
:100470000EF0E4A3F0A3F0A37411F0300505E4A39B
:10048000F0800690E74974FFF0000000E490E68AEF
:10049000F000000090E68B740AF012182802057034
:1004A00090E678E04480F090E6797491F07F647E85
:1004B0000012195790E679E090E740F07F647E00E3
:1004C00012195790E679E090E741F07F647E0012C0
:1004D000195790E679E090E742F07F647E001219A8
:1004E0005790E679E090E743F090E678E04440F0FA
:1004F000000000E490E68AF000000090E68B7404AF
:10050000F0806DE490E68AF090E68BF090E6A0E053
:1005100020E1F990E68BE0F55DD39401405290E73D
:1005200041E0FD7F4212185390E740E0FD7F4E12FC
:100530001853803CE490E68AF090E68BF090E6A0B9
:10054000E020E1F990E68BE0F55DD3940040219046
:10055000E740E07003121A8090E740E0B401031214
:100560001A8490E740E0B40207121AB28002D32244
:01057000C3C7
:010571002267
:10192700C0E0C083C082D2015391EF90E65D74019D
:08193700F0D082D083D0E03231
:10198500C0E0C083C0825391EF90E65D7404F0D04F
:0619950082D083D0E03295
:10199B00C0E0C083C0825391EF90E65D7402F0D03B
:0619AB0082D083D0E0327F
:10166A00C0E0C083C08290E680E030E70E85080CB7
:10167A0085090D85100E85110F800C85100C8511BA
:10168A000D85080E85090F5391EF90E65D7410F0F1
:07169A00D082D083D0E032C2
:10193F00C0E0C083C082D2035391EF90E65D74087C
:08194F00F0D082D083D0E03219
:1016A100C0E0C083C08290E680E030E70E85080C80
:1016B10085090D85100E85110F800C85100C851183
:1016C1000D85080E85090F5391EF90E65D7420F0AA
:0716D100D082D083D0E0328B
:011A90003223
:011A91003222
:011A92003221
:011A93003220
:1017A300C0E0C083C082C2AF90E7C0E53EF0000056
:1017B3000090E68F7404F00000005391EF90E65F11
:0D17C300E04404F0D2AFD082D083D0E032F9
:10106300C0E0C0F0C083C082C0D075D000C000C053
:0D10730001C002C003C004C005C006C007D4
:10108000C2AF90E6A1E020E1F990E780E0FF7004B4
:10109000F5238065BF011390E782E0F53590E78185
:1010A000E0F53A902746E4F0804FBF021C90E782BB
:1010B000E0902700F090E781E0902701F09027442E
:1010C000E4F0A3F0A304F08030BFFF07752300D243
:1010D000068026BFFE0890E781E0F540801B90E780
:1010E00082E0FD7F4212185390E781E0FD7F4E12AF
:1010F0001853E4FD7F9012185300000090E68DE431
:0D110000F05391EF90E65FE04408F0D2AFAD
:10110D00D007D006D005D004D003D002D001D00036
:0B111D00D0D0D082D083D0F0D0E032E0
:011A9400321F
:011A9500321E
:011A9600321D
:011A9700321C
:011A9800321B
:011A9900321A
:011A9A003219
:011A9B003218
:011A9C003217
:011A9D003216
:011A9E003215
:011A9F003214
:011AA0003213
:011AA1003212
:011AA2003211
:011AA3003210
:011AA400320F
:011AA500320E
:011AA600320D
:011AA700320C
:011AA800320B
:011AA900320A
:011AAA003209
:011AAB003208
:011AAC003207
:011AAD003206
:011AAE003205
:011AAF003204
:011AB0003203
:011AB1003202
:10195700AD07AC06ED25E0FDEC33FCED4C6007ED83
:071967001D70011C80F52238
:0612B8008C5F8D60A907A8
:1012BE00530107C2A77F0A7E00121957E4FBFAC337
:1012CE0074029BFFE9A807088002C313D8FC30E024
:1012DE0004D2A68002C2A67F0A7E00121957D2A59A
:1012EE00121957C2A51219570BBB00010AEB640362
:1012FE004A70CCE4FAFBC374099BFFE560AE5FA8AD
:10130E0007088005CEC313CE13D8F930E004D2A659
:10131E008002C2A67F0A7E00121957D2A512195753
:10132E00C2A51219570BBB00010AEB640A4A70C61C
:0E133E00D2A77F0A7E00121957C2A7121957B4
:01134C00227E
:0A1A0200AD07AC06E4FF1212B82293
:0A1A0C00AD07AC067F041212B822E9
:0A1A1600AD07AC067F051212B822DE
:0A1A2000AD07AC067F061212B822D3
:0A1A2A00AD07AC067F011212B822CE
:0A1A3400AD07AC067F021212B822C3
:0A1A3E00AD07AC067F031212B822B8
:0413D9008F62A90571
:1013DD00C2A47F017E00121957E4FBFAAF03E9A8FE
:1013ED0007088002C313D8FC30E004D2A68002C2E5
:1013FD00A67F017E00121957D2A5121957C2A51248
:10140D0019570BBB00010AEB64084A70CFE4FAFBD5
:10141D00AF03E562A807088002C313D8FC30E004CF
:10142D00D2A68002C2A67F017E00121957D2A51244
:10143D001957C2A51219570BBB00010AEB64084AD4
:10144D0070CEC2A4D2A47F017E00121957C2A4127D
:02145D0019571D
:01145F00226A
:041A780053B1FE2246
:041A7C0043B101224F
:071A580053B1FB43B1022270
:071A5F0043B10243B1042270
:071A660053B1FB53B1FD2257
:071A6D00121A7C121A5F221D
:10190D00121A7C000000121A587F3C7E00121957E3
:0A191D00121A5F121A7812195722ED
:1018C700121A587FAA7E00121957121A66121A7C2A
:1018D7007FC8121957121A78121A587F7812195797
:0418E700121A5F2250
:1015FB00E4F51CF51DE4FBFA12190D7F467E001273
:10160B0019570BBB00010ABA04EEBB06EBC28130C3
:10161B0080FDD281051DE51D7002051CC39404E5F8
:07162B001C6480948040CE96
:011632002295
:10154D00121A78121A5FE4F561F56243B1087F0F44
:10155D007E00121957E4FBFA121A7C121A587F14E6
:10156D007E00121957121A5F121A787F321219570C
:10157D000BBB00010AEB641E4A70DD53B1F77F14FB
:10158D007E00121957121A7C121A58121957121A74
:10159D005F121A780562E56270020561C39410E569
:0715AD00616480948140A4F9
:0115B4002214
:041A800043B18022CC
:041A840053B17F22B9
:0E00800053B1DF7F027E0012195743B12022D8
:100F9B00E4F563E52B452A7003120080E538B401B4
:100FAB0005D2081219E2E5367003121A80E5396092
:100FBB0003021048752301902704E075F040A485C7
:100FCB00F061F562AF237E00AC61AD62120B92D380
:100FDB00EF9400EE940040141211287F007E04124F
:100FEB0018EBE56215627002156180D8902705E059
:100FFB00756100F562AF237E00AC61AD62120B929E
:10100B00D3EF9400EE9400401E0563E563B406062F
:10101B00121128E4F5637F007E011218EBE56215CF
:10102B00627002156180CEE5636006121128E4F54B
:10103B0063902706E0FF7E001218EB8009752301F1
:10104B00E523640160FAE5367003121A84E538B4BF
:07105B000105C2081219E2B1
:01106200226B
:100C7C00C2A0C206753E02E52B452A70031218C7A6
:100C8C00E52B452A70031218C7E5417018120F9B0B
:100C9C00D2081219E2E52B452A700312154DC20831
:100CAC001219E2800CE52B452A700312154D120F18
:100CBC009B1218C730060412182822753E03E4F55F
:100CCC005DF55EC3E55E9528E55D95275029E4F555
:100CDC005FF560C3E56095347480F8655F98500DDE
:100CEC0012190D0560E5607002055F80E6055EE592
:100CFC005E7002055D80CCE537D3940040057F64BF
:100D0C0012187CE4F55DF55EC3E55E9546E55D95F0
:100D1C00455030C2813080FDD281E4F55FF560C36F
:100D2C00E56095347480F8655F98500D12190D05C7
:100D3C0060E5607002055F80E6055EE55E700205A9
:100D4C005D80C5E4F55DF55EC3E55E9543E55D95B7
:100D5C00425029E4F55FF560C3E56095347480F882
:100D6C00655F98500D12190D0560E5607002055F06
:100D7C0080E6055EE55E7002055D80CCE53CFD7F9E
:100D8C00401213D9E53DFD7F201213D9C28130806A
:100D9C00FDD281E52CFD7F401213D9E52DFD7F207E
:050DAC001213D9D2A0D2
:010DB100221F
:10185300AB05AE0790E678E04480F090E679EEF0D1
:101863007F647E00121957EBF012195790E678E067
:091873004440F07F641219572271
:011AB2002211
:10182800E4F561F562D2A07F327E001215B5C2A040
:101838007F327E001215B50562E56270020561C34C
:0A1848009403E5616480948040DBA6
:011852002273
:10187C008F61432904AD297F801213D9E561600B78
:10188C00C2813080FDD281156180F15329FBAD29D5
:06189C007F801213D92227
:10196E00E490E608F075C83443985053877FC2ACB4
:07197E0075CBFF75CA64225E
:0D19D500309902C2998F993099FDC2992274
:10177400E4F51EF51F209822051FE51F7002051EC3
:10178400AE1EFFE4FCFD7BFA7AFFF9F8C3120BDA14
:0E1794005004D2048004C20480DBC298AF99D6
:0117A2002224
:081A5000E4F51BD2E9D2AF223C
:1016D80090E678E020E6F9C2E990E678E04480F008
:1016E800EF25E090E679F090E678E030E0F990E6D2
:1016F80078E04440F090E678E020E6F990E678E07B
:0617080030E1D6D2E92217
:10174200A90790E678E020E6F9E51B702390E67899
:10175200E04480F0E925E090E679F08D16AF03A928
:10176200077517018A188919E4F51A751B01D32226
:02177200C32290
:10170E00A90790E678E020E6F9E51B702590E678CB
:10171E00E04480F0E925E0440190E679F08D16AFC3
:10172E0003A9077517018A188919E4F51A751B03A1
:04173E00D322C322CD
:03004B00020DB2F1
:100DB200C0E0C083C082C085C084C086758600C082
:100DC200D075D000C000C001C002C003C006C00779
:100DD20090E678E030E206751B06020E9C90E678FB
:100DE200E020E10CE51B64026006751B07020E9C05
:100DF200E51B24FE605F14603624FE7003020E8D34
:100E020024FC7003020E9924086003020E9CAB17A7
:100E1200AA18A919AF1A051A8F82758300120B43FB
:100E220090E679F0E51A65167070751B05806B9077
:100E3200E679E0AB17AA18A919AE1A8E827583005B
:100E4200120B70751B02E5166401704E90E678E095
:100E52004420F08045E51624FEB51A0790E678E0B6
:100E62004420F0E51614B51A0A90E678E04440F002
:100E7200751B0090E679E0AB17AA18A919AE1A8E75
:100E820082758300120B70051A800F90E678E04499
:100E920040F0751B008003751B005391DFD007D013
:100EA20006D003D002D001D000D0D0D086D084D0DA
:080EB20085D082D083D0E0322C
:0300000002134D9B
:0C134D00787FE4F6D8FD758165021394EA
:100B4300BB010CE58229F582E5833AF583E0225067
:100B530006E92582F8E622BBFE06E92582F8E222B1
:0D0B6300E58229F582E5833AF583E49322CB
:100B7000F8BB010DE58229F582E5833AF583E8F0BB
:100B8000225006E92582C8F622BBFE05E92582C867
:020B9000F2224F
:100B9200EF8DF0A4A8F0CF8CF0A428CE8DF0A42E77
:020BA200FE2231
:100BA400C2D5EC30E709B2D5E4C39DFDE49CFCEE6C
:100BB40030E715B2D5E4C39FFFE49EFE120C27C3B1
:100BC400E49DFDE49CFC8003120C2730D507C3E4AC
:060BD4009FFFE49EFE22DB
:100BDA00EB9FF5F0EA9E42F0E99D42F0EC6480C892
:060BEA0064809845F02232
:100BF000EB9FF5F0EA9E42F0E99D42F0E89C45F05B
:010C000022D1
:100C0100D083D082F8E4937012740193700DA3A382
:100C110093F8740193F5828883E473740293686096
:060C2100EFA3A3A380DF96
:1013590002080CE493A3F8E493A34003F68001F296
:1013690008DFF48029E493A3F85407240CC8C33395
:10137900C4540F4420C8834004F456800146F6DF64
:10138900E4800B0102040810204080901460E47E80
:10139900019360BCA3FF543F30E509541FFEE49359
:1013A900A360010ECF54C025E060A840B8E493A320
:1013B900FAE493A3F8E493A3C8C582C8CAC583CA4B
:1013C900F0A3C8C582C8CAC583CADFE9DEE780BE03
:0114DF00000C
:100C2700BC000BBE0029EF8DF084FFADF022E4CCB1
:100C3700F875F008EF2FFFEE33FEEC33FCEE9DEC7A
:100C4700984005FCEE9DFE0FD5F0E9E4CEFD22EDC0
:100C5700F8F5F0EE8420D21CFEADF075F008EF2F0A
:100C6700FFED33FD4007985006D5F0F222C398FDFB
:050C77000FD5F0EA2298
:00000001FF
